:020000040000FA
:0400000023EF00F0FA
:020004000000FA
:040008000FEF00F006
:040018000FEF00F0F6
:04001C001000006E62
:10002000D838016EF2B402D01CEF00F05986162EBB
:1000300003D05A84640E166E0138D86E003A003828
:10004000F294F28E100066EC01F0566AF29EF29A7B
:10005000F2949FEC0AF0A3EC07F09488948C9380C0
:100060008A988B8A78EC07F078EC07F082A809D0A0
:100070008B9A78EC07F078EC07F082B802D05990B0
:1000800001D059808B9A8B8E78EC07F078EC07F0D2
:1000900082AC09D08B9E78EC07F078EC07F082BC3C
:1000A00002D0599201D059828B9E8A8278EC07F057
:1000B00078EC07F081A009D08A9278EC07F078EC10
:1000C00007F081B002D0599401D059848A9266EC2D
:1000D00001F04AEC0AF093EC07F029EC0BF088EC05
:1000E00009F093EC07F029EC0BF0C8EC09F093EC65
:1000F00007F029EC0BF0F0EC09F0F6EC01F029EC3C
:100100000BF009EC09F093EC07F029EC0BF056EC3E
:1001100008F059A401D003D0080E4B6E03D0040E92
:100120004B6E00D059A201D003D0040E4A6E03D00A
:10013000020E4A6E00D0F28E010EC26E2FEC04F059
:1001400060C00FF05FC00EF0050EC26E2FEC04F021
:1001500060C011F05FC010F059B036D00FC009F088
:100160000EC008F011C007F010C006F01250085E73
:100170001350095AD8B003D0096A086A0ED00F0E7E
:10018000096401D006D0096206D0A00E086403D02D
:1001900000D0598C02D0599C00D01450065E1550E6
:1001A000075AD8B003D0076A066A44D00F0E076416
:1001B00001D006D0076206D0A00E066403D000D09E
:1001C000598A38D0599A36D00FC007F00EC006F0C1
:1001D00011C009F010C008F01250065E1350075A03
:1001E000D8B003D0076A066A0ED00F0E076401D09C
:1001F00006D0076206D0A00E066403D000D0598A4C
:1002000002D0599A00D01450085E1550095AD8B03F
:1002100003D0096A086A0ED00F0E096401D006D017
:10022000096206D0A00E086403D000D0598C02D019
:10023000599C00D059B60CD05AB4F6EC01F09AECA7
:1002400005F089EC01F080AC76D71EEC02F073D794
:10025000599607C002F006C003F01BEC05F017C06A
:1002600038F018C039F019C03AF01AC03BF009C094
:1002700002F008C003F01BEC05F017C03CF018C0FA
:100280003DF019C03EF01AC03FF00BC002F00AC0AA
:1002900003F01BEC05F017C040F018C041F019C086
:1002A00042F01AC043F058EC06F05BEC03F0BDECF2
:1002B00003F080AC01D005D081EC02F0DFEC02F05D
:1002C0003AD71EEC02F037D764EF01F07C0ED36E04
:1002D0009B8C000E936E020E946E4F0E926E8A6A85
:1002E0008B6A898E0C0EBD6E040ECA6EFF0ECB6E2D
:1002F000000EBE6EBD9ABD98010EC26E3B0EC16E61
:100300008D0EC06E950ED56EF26AF28EF28AF28C68
:1003100012000BC06FF00AC06EF0270E716E100E47
:10032000706E56EC05F075C069F074C068F073C06B
:1003300067F072C066F059A201D003D059A404D06E
:1003400011D059A408D015D03D0E636E180E626E00
:1003500077EC05F015D04C0E636E5E0E626E77EC96
:1003600005F00ED0980E636EBC0E626E77EC05F051
:1003700007D0BE0E636EEB0E626E77EC05F000D018
:10038000080E4C6207D0000E636E640E626E77EC4E
:1003900005F00AD0040E4C6207D0000E636E0A0E00
:1003A000626E77EC05F000D0030E676401D006D0D2
:1003B000676209D0FF0E666406D000D0030E676E38
:1003C000FF0E666E00D066A002D0BD8801D0BD9839
:1003D00066A202D0BD8A01D0BD9AD890673266323B
:1003E000D8906732663266C0BEFF12008B8683ECFF
:1003F00007F083EC07F083EC07F083EC07F083EC65
:1004000007F0010EC26E2FEC04F060C013F05FC065
:1004100012F0050EC26E2FEC04F060C015F05FC044
:1004200014F08B9683EC07F083EC07F083EC07F075
:1004300083EC07F083EC07F05A94120059AC34D0E7
:10044000400EF1EC0AF0050EC8EC0AF0050EC8ECFF
:100450000AF0050EC8EC0AF0050EC8EC0AF0050E0D
:10046000C8EC0AF0050EC8EC0AF0050EC8EC0AF05C
:10047000050EC8EC0AF0050EC8EC0AF0050EC8EC33
:100480000AF0050EC8EC0AF0050EC8EC0AF0050EDD
:10049000C8EC0AF0050EC8EC0AF0050EC8EC0AF02C
:1004A000050EC8EC0AF01200400EF1EC0AF0506A9A
:1004B00009C04FF008C04EF0100E516EFA0E4E5C9F
:1004C000D8B001D006D04E6E050EC8EC0AF0510629
:1004D000F5D74F06D8B0F7D700D04F6A320E4E5E30
:1004E000D8B001D002D0502AF8D75050C8EC0AF04A
:1004F0005106516601D01200200EC8EC0AF0F8D760
:100500001200000E4C6204D0410EF1EC0AF004D04F
:10051000400EF1EC0AF000D0406606D04CB604D094
:10052000200EC8EC0AF004D0300E4024C8EC0AF0CB
:100530004CA604D02E0EC8EC0AF000D041660AD0BA
:100540004CB608D04CB406D0406604D0200EC8EC9F
:100550000AF004D0300E4124C8EC0AF04CA404D0B8
:100560002E0EC8EC0AF000D042660ED04CB60CD06D
:100570004CB40AD04CB208D0406606D0416604D0D4
:10058000200EC8EC0AF004D0300E4224C8EC0AF069
:100590004CA204D02E0EC8EC0AF000D0300E43243A
:1005A000C8EC0AF0570EC8EC0AF0200EC8EC0AF0AE
:1005B000200EC8EC0AF0200EC8EC0AF012005AA077
:1005C00019D0490EF1EC0AF0200EC8EC0AF02D0EFD
:1005D000C8EC0AF02D0EC8EC0AF02D0EC8EC0AF09B
:1005E0002D0EC8EC0AF06B0EC8EC0AF0060EC8EC33
:1005F0000AF01200000E4D6204D04A0EF1EC0AF02F
:1006000004D0490EF1EC0AF000D0446606D04DB695
:1006100004D0200EC8EC0AF004D0300E4424C8ECFC
:100620000AF04DA604D02E0EC8EC0AF000D04566A4
:100630000AD04DB608D04DB406D0446604D0200E82
:10064000C8EC0AF004D0300E4524C8EC0AF04DA4E2
:1006500004D02E0EC8EC0AF000D046660ED04DB67F
:100660000CD04DB40AD04DB208D0446606D04566D1
:1006700004D0200EC8EC0AF004D0300E4624C8EC9A
:100680000AF04DA204D02E0EC8EC0AF000D0300EB5
:100690004724C8EC0AF059A807D06B0EC8EC0AF042
:1006A000060EC8EC0AF01200060EC8EC0AF0200E86
:1006B000C8EC0AF01200000EF1EC0AF059AA13D0AF
:1006C000200EC8EC0AF02D0EC8EC0AF02D0EC8EC76
:1006D0000AF02D0EC8EC0AF02D0EC8EC0AF0560EEA
:1006E000C8EC0AF01200386606D04AB604D0200ED4
:1006F000C8EC0AF004D0300E3824C8EC0AF04AA640
:1007000004D02E0EC8EC0AF000D039660AD04AB6E2
:1007100008D04AB406D0386604D0200EC8EC0AF0DF
:1007200004D0300E3924C8EC0AF04AA404D02E0EAE
:10073000C8EC0AF000D03A660ED04AB60CD04AB4E3
:100740000AD04AB208D0386606D0396604D0200EE6
:10075000C8EC0AF004D0300E3A24C8EC0AF04AA2E1
:1007600004D02E0EC8EC0AF000D0300E3B24C8ECAA
:100770000AF0560EC8EC0AF01200090EF1EC0AF06D
:1007800059AC16D0200EC8EC0AF02D0EC8EC0AF0B9
:100790002D0EC8EC0AF02D0EC8EC0AF02D0EC8EC98
:1007A0000AF0410EC8EC0AF0200EC8EC0AF0120064
:1007B0003C6606D04BB604D0200EC8EC0AF004D03C
:1007C000300E3C24C8EC0AF04BA604D02E0EC8EC28
:1007D0000AF000D03D660AD04BB608D04BB406D024
:1007E0003C6604D0200EC8EC0AF004D0300E3D2444
:1007F000C8EC0AF04BA404D02E0EC8EC0AF000D0CE
:100800003E660ED04BB60CD04BB40AD04BB208D0DB
:100810003C6606D03D6604D0200EC8EC0AF004D039
:10082000300E3E24C8EC0AF04BA204D02E0EC8ECC9
:100830000AF000D0300E3F24C8EC0AF0020E4B62E2
:1008400007D06D0EC8EC0AF0410EC8EC0AF0120099
:10085000410EC8EC0AF0200EC8EC0AF01200500E4F
:100860005B6E01EE00F0C28062EC07F0C282C2B2A1
:1008700037EF04F0C3CFEEFFC4CFEEFF5B2EF6D709
:100880005C6A01EE01F011EE03F0EF50E76401D075
:100890001BD0E76209D0ED52E552EF50E76401D07A
:1008A00018D0E652EE5200D0E652E652010EE26255
:1008B0002CD0A10EE162E9D700D0ED6AEE6A5C2A85
:1008C000080E5C62DED70CD0E1CFE9FFE2CFEAFF91
:1008D000EBD7E1CFE9FFE2CFEAFFEE52E652E4D7F1
:1008E0005C6A01EE01F011EE03F0EF660ED0ED52FE
:1008F000EE660BD0EE52EE52E652E652010EEA627E
:10090000F4D79F0EE962F1D70ED0E76613D0E55217
:10091000E66610D0E652E652010EE262F6D7A10E6C
:10092000E162F3D700D0ED6AEE6A5C2A080E5C62E1
:10093000D8D71BD0EF50E76001D00BD0E762EAD7E1
:10094000ED52E552EF50E76001D008D0E652EE528A
:10095000E1D7E1CFE9FFE2CFEAFFDCD7E1CFE9FF62
:10096000E2CFEAFFEE52E652D5D75F6A606A616A6B
:10097000500E5C6E01EE00F0EE505F26EE506022ED
:10098000D8A001D0612A5C065C66F6D7200E5F26EF
:10099000000E6022000E6122D890613260325F3218
:1009A000D890613260325F32D890613260325F320B
:1009B000D890613260325F32D890613260325F32FB
:1009C000D890613260325F32120030D8F36ED89026
:1009D0000BD020EE20F0330EDF26DFB6F00BDFBEAB
:1009E0000F0BDE5ED9A4F7D72536263627362036FC
:1009F000213622362336F32EECD723380F0B2F6EF9
:100A000023500F0B2E6E22380F0B2D6E22500F0B22
:100A10002C6E21380F0B2B6E21500F0B2A6E2038B5
:100A20000F0B296E20500F0B286E1200206A216ACE
:100A3000226A236A180C176A186A196A1A6A030E5E
:100A4000025CE80ED8B4035CD8A039EF05F0030EC1
:100A5000025CD8A039EF05F030EF05F039EF05F072
:100A6000026EE80E035C036ED8A00206172A1FEF81
:100A700005F0640E035CD8B044EF05F0026642EF67
:100A800005F048EF05F00206036E182A39EF05F06D
:100A90000A0E035CD8A053EF05F0192A036E48EF45
:100AA00005F003C01AF003C01AF01200726A736AEC
:100AB000746A756A70506E02F3CF72F0F4CF73F0FF
:100AC00071506F02F3CF74F0F4CF75F070506F0275
:100AD000F3507326F4507422E86A752271506E0246
:100AE000F3507326F4507422E86A75221200200E27
:100AF0006A6E656A646AD8906636673668366936A3
:100B000064366536D8B08FEF05F06350655CD8A4C5
:100B10008CEF05F06250645CD8A096EF05F062504F
:100B2000645ED8A065066350655E66806A2E7BEFC2
:100B300005F0120007C06FF006C06EF009C071F03A
:100B400008C070F056EC05F07F0E6A6E960E6B6E64
:100B5000980E6C6E000E6D6E72506A5C73506B581E
:100B600074506C5875506D5801E207D0080E4A62F7
:100B700051D0020E4B624ED000D0880E7226130E5A
:100B80007322000E7422000E7522100E626E270E64
:100B9000636E72C066F073C067F074C068F075C0B1
:100BA00069F077EC05F067C00BF066C00AF0080E3C
:100BB0004A620FD0020E4B6203D0080E4C6E77D003
:100BC000080E4B6203D0040E4C6E71D0020E4C6EB8
:100BD0006ED0040E4A620FD0020E4B6203D0040E98
:100BE0004C6E65D0080E4B6203D0020E4C6E5FD087
:100BF000020E4C6E5CD0020E4B6203D0020E4C6EA5
:100C000056D0080E4B6203D0020E4C6E50D0000E30
:100C10004C6E4DD0F40E7226010E7322000E74221B
:100C2000000E7522E80E626E030E636E72C066F0EF
:100C300073C067F074C068F075C069F077EC05F0B8
:100C400067C00BF066C00AF0080E4A620FD0020EB1
:100C50004B6203D0080E4C6E2AD0080E4B6203D0B4
:100C6000080E4C6E24D0040E4C6E21D0040E4A6245
:100C70000FD0020E4B6203D0080E4C6E18D0080E37
:100C80004B6203D0040E4C6E12D0020E4C6E0FD08D
:100C9000020E4B6203D0040E4C6E09D0080E4B625C
:100CA00003D0020E4C6E03D0000E4C6E00D012002A
:100CB000096604D0086602D05A8012005A905998EA
:100CC000100E4D6E080E4A6204D04D464D464D46FC
:100CD0000BD0040E4A6203D04D464D4605D0020E9D
:100CE0004A6202D04D4600D0080E4B6204D04D42FD
:100CF0004D424D420ED0040E4B6203D04D424D4248
:100D000008D0020E4B62FDD74D424D424D424D423E
:100D100000D007C06FF006C06EF0270E716E100E87
:100D2000706E56EC05F0800E4D6201D00CD0400E76
:100D30004D6201D023D0200E4D6201D039D0100E6B
:100D40004D6267D04ED0270E636E100E626E72C079
:100D500066F073C067F074C068F075C069F077EC36
:100D600005F066C072F067C073F068C074F069C0C7
:100D700075F04D424D424D424D424BD0030E636ED5
:100D8000E80E626E72C066F073C067F074C068F0FF
:100D900075C069F077EC05F066C072F067C073F05B
:100DA00068C074F069C075F04D424D424D4231D07B
:100DB000000E636E640E626E72C066F073C067F000
:100DC00074C068F075C069F077EC05F066C072F029
:100DD00067C073F068C074F069C075F04D424D4251
:100DE00018D0000E636E0A0E626E72C066F073C099
:100DF00067F074C068F075C069F077EC05F066C004
:100E000072F067C073F068C074F069C075F04D424D
:100E100000D009C063F008C062F072C066F073C011
:100E200067F074C068F075C069F077EC05F068C0D1
:100E300027F067C026F066C025F0E5EC04F02F66C9
:100E400001D00BD02FC044F02EC045F02DC046F08D
:100E50002CC047F04D42598834D02E6601D00AD0BC
:100E60002EC044F02DC045F02CC046F02BC047F0FA
:100E7000598827D02D6601D00CD02DC044F02CC04D
:100E800045F02BC046F02AC047F04D424D425998DC
:100E900018D02C6601D00BD02CC044F02BC045F0EC
:100EA0002AC046F029C047F04D4259980AD02BC0BD
:100EB00044F02AC045F029C046F028C047F05998B0
:100EC00000D01200020E546E290E536E532E66EFA0
:100ED00007F0542E66EF07F012000C0E546EAE0EA3
:100EE000536E532E71EF07F0542E71EF07F012007E
:100EF000750E546EE00E536E532E7CEF07F0542E99
:100F00007CEF07F01200050E556E910E546ECF0E59
:100F1000536E532E89EF07F0542E89EF07F0552EAC
:100F200089EF07F012002E0E556EA90E546E2E0E8C
:100F3000536E532E99EF07F0542E99EF07F0552E6C
:100F400099EF07F0120029EC0BF0400E0EEC0BF0BD
:100F5000000EC8EC0AF00A0EC8EC0AF0000EC8EC4D
:100F60000AF00E0EC8EC0AF0110EC8EC0AF0110ED1
:100F7000C8EC0AF00E0EC8EC0AF0000EC8EC0AF03D
:100F8000020EC8EC0AF0040EC8EC0AF00E0EC8EC13
:100F90000AF0110EC8EC0AF01F0EC8EC0AF0100E91
:100FA000C8EC0AF00E0EC8EC0AF0000EC8EC0AF00D
:100FB000020EC8EC0AF0040EC8EC0AF0000EC8ECF1
:100FC0000AF00C0EC8EC0AF0040EC8EC0AF0040E8D
:100FD000C8EC0AF00E0EC8EC0AF0000EC8EC0AF0DD
:100FE000050EC8EC0AF00A0EC8EC0AF0000EC8ECB8
:100FF0000AF00E0EC8EC0AF0110EC8EC0AF0110E41
:10100000C8EC0AF00E0EC8EC0AF0000EC8EC0AF0AC
:101010000A0EC8EC0AF0000EC8EC0AF0110EC8EC7B
:101020000AF0110EC8EC0AF0110EC8EC0AF0110E0D
:10103000C8EC0AF00E0EC8EC0AF0000EC8EC0AF07C
:10104000020EC8EC0AF0040EC8EC0AF0000EC8EC60
:101050000AF00E0EC8EC0AF0110EC8EC0AF0110EE0
:10106000C8EC0AF00E0EC8EC0AF0000EC8EC0AF04C
:10107000020EC8EC0AF0040EC8EC0AF00E0EC8EC22
:101080000AF0110EC8EC0AF01F0EC8EC0AF0110E9F
:10109000C8EC0AF0110EC8EC0AF0000EC8EC0AF019
:1010A000000EF1EC0AF029EC0BF0120029EC0BF029
:1010B000400E0EEC0BF0000EC8EC0AF0000EC8EC6F
:1010C0000AF0000EC8EC0AF0000EC8EC0AF0000EA0
:1010D000C8EC0AF0000EC8EC0AF0000EC8EC0AF0EA
:1010E000000EC8EC0AF0100EC8EC0AF0100EC8ECA6
:1010F0000AF0100EC8EC0AF0100EC8EC0AF0100E40
:10110000C8EC0AF0100EC8EC0AF0100EC8EC0AF099
:10111000100EC8EC0AF0180EC8EC0AF0180EC8EC55
:101120000AF0180EC8EC0AF0180EC8EC0AF0180EF7
:10113000C8EC0AF0180EC8EC0AF0180EC8EC0AF059
:10114000180EC8EC0AF01C0EC8EC0AF01C0EC8EC15
:101150000AF01C0EC8EC0AF01C0EC8EC0AF01C0EBB
:10116000C8EC0AF01C0EC8EC0AF01C0EC8EC0AF021
:101170001C0EC8EC0AF01E0EC8EC0AF01E0EC8ECDD
:101180000AF01E0EC8EC0AF01E0EC8EC0AF01E0E85
:10119000C8EC0AF01E0EC8EC0AF01E0EC8EC0AF0ED
:1011A0001E0EC8EC0AF01F0EC8EC0AF01F0EC8ECA9
:1011B0000AF01F0EC8EC0AF01F0EC8EC0AF01F0E52
:1011C000C8EC0AF01F0EC8EC0AF01F0EC8EC0AF0BB
:1011D0001F0EC8EC0AF0000EC8EC0AF0000EC8ECB6
:1011E0000AF00E0EC8EC0AF0110EC8EC0AF0110E4F
:1011F000C8EC0AF00A0EC8EC0AF01B0EC8EC0AF0A4
:10120000000EC8EC0AF0000EF1EC0AF029EC0BF02D
:10121000120013C002F012C003F01BEC05F019C05D
:101220001CF01AC01DF015C002F014C003F01BEC36
:1012300005F019C01EF01AC01FF0000EF1EC0AF004
:10124000410EC8EC0AF04E0EC8EC0AF0300EC8ECA5
:101250000AF0200EC8EC0AF06F0EC8EC0AF0660E19
:10126000C8EC0AF0660EC8EC0AF0730EC8EC0AF07F
:10127000650EC8EC0AF0740EC8EC0AF03A0EC8EC21
:101280000AF0200EC8EC0AF01C50300FC8EC0AF02F
:101290001D50300FC8EC0AF06D0EC8EC0AF0560E67
:1012A000C8EC0AF0400EF1EC0AF0410EC8EC0AF06E
:1012B0004E0EC8EC0AF0310EC8EC0AF0200EC8EC55
:1012C0000AF06F0EC8EC0AF0660EC8EC0AF0660E63
:1012D000C8EC0AF0730EC8EC0AF0650EC8EC0AF010
:1012E000740EC8EC0AF03A0EC8EC0AF0200EC8ECF6
:1012F0000AF01E50300FC8EC0AF01F50300FC8EC37
:101300000AF06D0EC8EC0AF0560EC8EC0AF0120096
:10131000000EF1EC0AF0500EC8EC0AF0490EC8ECD1
:101320000AF0430EC8EC0AF02D0EC8EC0AF0650E68
:10133000C8EC0AF0730EC8EC0AF0200EC8EC0AF0F4
:10134000700EC8EC0AF0610EC8EC0AF06E0EC8EC24
:101350000AF0650EC8EC0AF06C0EC8EC0AF06D0ECF
:10136000C8EC0AF0010EC8EC0AF0720EC8EC0AF0E4
:10137000030EC8EC0AF0470EF1EC0AF0490EC8EC77
:101380000AF0490EC8EC0AF02E0EC8EC0AF0120062
:10139000420EF1EC0AF0760EC8EC0AF0650EC8ECCD
:1013A0000AF0720EC8EC0AF07A0EC8EC0AF0690E68
:1013B000C8EC0AF0050EC8EC0AF03A0EC8EC0AF0C8
:1013C000010E300FC8EC0AF02E0EC8EC0AF0010E28
:1013D000300FC8EC0AF0000E300FC8EC0AF0120013
:1013E000010EF1EC0AF0700EC8EC0AF0610EC8ECC8
:1013F0000AF02D0EC8EC0AF0650EC8EC0AF06C0E6F
:10140000C8EC0AF0650EC8EC0AF06B0EC8EC0AF0E6
:10141000740EC8EC0AF0720EC8EC0AF06F0EC8EC3D
:101420000AF06E0EC8EC0AF0690EC8EC0AF06B0EFA
:10143000C8EC0AF0610EC8EC0AF0430EF1EC0AF0B9
:10144000020E300FC8EC0AF0000E300FC8EC0AF0A4
:10145000010E300FC8EC0AF0000E300FC8EC0AF095
:101460002E0EC8EC0AF0000E300FC8EC0AF0080E81
:10147000300FC8EC0AF02E0EC8EC0AF0010E300F47
:10148000C8EC0AF0020E300FC8EC0AF02E0EC8ECC1
:101490000AF01200410EC8EC0AF0640EC8EC0AF023
:1014A0006A0EC8EC0AF06F0EC8EC0AF06E0EC8ECBB
:1014B0000AF0200EC8EC0AF0610EC8EC0AF07A0EB1
:1014C000C8EC0AF0200EC8EC0AF0490EC8EC0AF08D
:1014D000730EC8EC0AF0740EC8EC0AF0650EC8EC86
:1014E0000AF06E0EC8EC0AF02C0EC8EC0AF0420EA0
:1014F000F1EC0AF0730EC8EC0AF07A0EC8EC0AF0B0
:10150000650EC8EC0AF0620EC8EC0AF0620EC8EC78
:101510000AF0200EC8EC0AF06A0EC8EC0AF0000EC1
:10152000C8EC0AF0760EC8EC0AF0030EC8EC0AF01C
:10153000740EC8EC0AF0210EC8EC0AF0120083EC1D
:1015400007F083EC07F083EC07F083EC07F083EC03
:1015500007F08A9A8A988B988B9A8B9C8B9E8A80AC
:101560008A828A948A9678EC07F08A8878EC07F069
:101570008A988B988B9A8B8C8B8E8A808A828A949D
:101580008A9678EC07F08A8878EC07F08A9812003F
:10159000F2AE01D002D05A9201D05A82F29E8A98BD
:1015A0008A8A8A968A948A928A908B9E8B9C8B9A3E
:1015B0008B98E8B08A86E8B28A84E8B48A82E8B672
:1015C0008A80E8B88B8EE8BA8B8CE8BC8B8AE8BE40
:1015D0008B888A8862EC07F08A985AA21200F28EF1
:1015E00012008A988A9A8A968A948A928A908B9E06
:1015F0008B9C8B9A8B88E8B08A86E8B28A84E8B4A0
:101600008A82E8B68A80E8B88B8EE8BA8B8CE8BC10
:101610008B8A8A8862EC07F08A9812008A988A9AE4
:101620008A968A948A928A908B9E8B9C8B8A8B98BE
:10163000E8B08A86E8B28A84E8B48A82E8B68A800A
:10164000E8B88B8EE8BA8B8C8A8862EC07F08A98AF
:1016500012008A988A9A8A868A948A928A908B9EA5
:101660008B9C8B9A8B988A8862EC07F08A986DEC39
:1016700007F06DEC07F01200000EF1EC0AF0200EFE
:10168000C8EC0AF0C8EC0AF0C8EC0AF0C8EC0AF0A2
:10169000C8EC0AF0C8EC0AF0C8EC0AF0C8EC0AF092
:1016A000C8EC0AF0C8EC0AF0C8EC0AF0C8EC0AF082
:1016B000C8EC0AF0C8EC0AF0C8EC0AF0C8EC0AF072
:1016C0001200400EF1EC0AF0200EC8EC0AF0C8EC53
:1016D0000AF0C8EC0AF0C8EC0AF0C8EC0AF0C8EC52
:1016E0000AF0C8EC0AF0C8EC0AF0C8EC0AF0C8EC42
:1016F0000AF0C8EC0AF0C8EC0AF0C8EC0AF0C8EC32
:101700000AF0C8EC0AF0C8EC0AF0120086EF0BF001
:020000040030CA
:0100010038C6
:01000200F904
:01000300FEFE
:010005007B7F
:01000600BB3E
:01000800FCFB
:01000900BF37
:01000A00FFF6
:01000B00FFF5
:01000C00FFF4
:01000D00FFF3
:00000001FF
